:03000000023D9A24
:0C3D9A0078FFE4F6D8FD75816A023DE177
:101B200020000A3C2E2E2E3E004950436F6E6E65FB
:101B300063745245510A004950436F6E6E65637479
:101B4000000A49504E6F41434B210A003E432C5638
:101B50002C43432CC0E4E0EFF2E5F020D1E8EDEABD
:101B6000EEEC49500A003E432C4D41432C253032C7
:101B700062583A25303262583A25303262583A2556
:101B8000303262583A25303262583A253032625843
:101B90002C4D414320E0E4F0E5F10A003E432C5691
:101BA00045522C20332E3220EEF22025732025734F
:101BB0002CC2E5F0F1E8FF20495020ECEEE4F3EB15
:101BC000FF0A004A756E203234203230303800313E
:101BD000363A30343A3033003E432C4C442C505289
:101BE0004F473A2020202020202020202020202085
:101BF00020202020202020202020202020202020E5
:101C000020202020202020202020202020202020D4
:101C100020202020202020202020202020202020C4
:101C200020202020202020202CC4E0F2E020EFF013
:101C3000EEF8E8E2EAE828F4E0E9EB290A003E2AB7
:101C40002C312CCEF1EDEEE2EDFBE520EFE0F0E003
:101C5000ECE5F2F0FB20F1E5F2E5E2EEE3EE20E860
:101C6000EDF2E5F0F4E5E9F1E00A003E412C413007
:101C7000312C2562752E2562752E2562752E256202
:101C8000752C495020E0E4F0E5F120E0E4E0EFF2CB
:101C9000E5F0E00A003E412C4130322C2562752EE1
:101CA0002562752E2562752E2562752C495020E01F
:101CB000E4F0E5F120EEF1ED2E20F1E5F0E2E5F0C3
:101CC000E00A003E412C4130332C2562752E2562FE
:101CD000752E2562752E2562752C495020E0E4F0A2
:101CE000E5F120F0E5E72E20F1E5F0E2E5F0E00A8D
:101CF000003E412C4130342C2562752E2562752E14
:101D00002562752E2562752CCCE0F1EAE020F1E524
:101D1000F2E80A003E412C4130352C2562752E2513
:101D200062752E2562752E2562752CD8EBFEE70AAA
:101D3000003E2A2C312CC4EEEF2E20EFE0F0E0EC38
:101D4000E5F2F0FB20F1E5F2E5E2EEE3EE20E8ED6E
:101D5000F2E5F0F4E5E9F1E00A003E422C533031BF
:101D60002C2562752CC6E4E0F2FC20E7E0EFF0EEF3
:101D7000F1E020F1EEE5E4E8EDE5EDE8FF20EEF23C
:101D800020F1E5F0E2E5F0E00A003E422C5330326B
:101D90002C2562752CCEE1ECE5ED20F120F1E5F08B
:101DA000E2E5F0EEEC20E1E5E720EAE2E8F2E0ED42
:101DB000F6E8E90A003E422C5330332C2562752C9C
:101DC000CFE5F0E5E7E0EFF3F1EA20EFF0E820EF10
:101DD000EEF2E5F0E520F1E2FFE7E820F120F1E5A1
:101DE000F0E2E5F0EEEC0A003E454E440A000A44FB
:101DF000756D705820202020203030203031203068
:101E00003220303320303420303520303620303707
:101E100020303820303920304120304220304320DB
:101E20003044203045203046000A3A003A20000A6B
:101E3000000A44756D70442020202020303020306E
:101E400031203032203033203034203035203036CD
:101E500020303720303820303920304120304220A7
:101E600030432030442030452030460045727220F7
:101E70006B657900526420656570726F6D0A00525F
:101E800064204D454D0A00526420436F64650A008A
:101E9000577269746520436F64650A004465627512
:101EA000674950204F4E0A004465627567495020CB
:101EB0004F46460A00446562756755736572204F48
:101EC0006E0A00446562756755736572204F464619
:101ED0000A0044656275674D7367204F6E0A0044BF
:101EE000656275674D7367204F46460A00436F6E03
:101EF000666967206C6F636B210A00577220656505
:101F000070726F6D0A00205361766520656570728E
:101F10006F6D210A00457272204D414321004C6FC4
:101F200061643E3E002A003C4130313D003C41307E
:101F3000323D003C4130333D003C4130343D003CBB
:101F40004130353D003C21003C5330313D003C5395
:101F500030323D003C5330333D003C5330353D0082
:061F60003C5330363D0049
:0647E200010B00010900BB
:10482B00C28E438910758BFF758DB7D2ABD28E229A
:03001B00023C7C28
:103C7C00C0E0C083C082C0D0C28E758BFF758DB77B
:103C8C0020060675A61E75A6E10509D202E50B6095
:103C9C0002050BE50AD394014002150A050EE50E48
:103CAC00540F7048D20EE50E543F7012D20090663D
:103CBC008BE0600A04F0E0D394B44002D206906624
:103CCC0086E0600204F0906104E0600214F09066FB
:103CDC008CE0D394014003E014F0300502050CE5B0
:103CEC000DD394644004D2068002050DE508D394EC
:103CFC000140021508D28ED0D0D082D083D0E032D1
:10105300C2AFC291C290D2B5C20B7D027C007F07A2
:101063001247C58F24E524646060097D017F601207
:101073004760D20BE4FDFC7F0B1247C58F24E524A8
:1010830030E6097D04E4FF124784D20B7D017C0026
:101093007F071247C58F24E5247008FD7FFF1247A1
:1010A30060D20B300B03126000C288C2A8C2AA75BB
:1010B30089001240C290633EE0B4FA06A3E064CE16
:1010C300607BE4F52474362524F582E43463F583E8
:1010D300E4F00524E524B443EC90633E74FAF0A3F2
:1010E30074CEF0A374CCF0906344740AF0E4A3F0DC
:1010F300A304F0A3F090633A74FFF0A3F0A3F0E429
:10110300A3F0906355740AF0E4F524E5242401FF69
:10111300E433FE74362524F582E43463F583E0FD7D
:1011230012473C0524E524C3944340DFE4F5A77547
:10113300A61E75A6E1907FF0F0A3F080FE906349B0
:101143007403F0A374CCF0E4906348F01239A4C2A2
:10115300B5124234C2061245C6D20BC20DC20C9060
:1011630065767408F09062B47424F0E4A3F090639D
:101173003EE09062B6F090633FE09062B7F0906318
:1011830040E09062B8F0906341E09062B9F0906300
:1011930042E09062BAF0906343E09062BBF0750A5C
:1011A30001E4906577F0C207C208C209C20A200BA6
:1011B30018AF24FE7D0312370CE4FF123A6E7E1B38
:1011C3007F20E4FBFDFC12324390668BE0600374E6
:1011D30001F0E4906104F0F50C906575F0F50D12E3
:1011E300482B75A70775A61E75A6E1D2AFE4F50DCA
:1011F300906104E07003121F6690668CE0B40111E5
:101203009080007410F0E490668CF0D20BC20CC294
:101213000D908008E0F52430E405D2077410F0E562
:101223002430E508D2099080087420F0E52430E6E4
:1012330008D2089080087440F0E50CC39403401969
:10124300908002E4F0908001F0908000F0E50C942F
:10125300064006E4F50C1245C69080A0E070031228
:1012630041409080B8E070031241BA9080D0E070A2
:101273000312456A908000E0701330071012334A5E
:10128300906331EFF0D39400400312002690800264
:10129300E07006908000E06005D2050211F0C205FF
:1012A300E4F50C906104E060030211F0200B12904E
:1012B3006578E0600C7E1B7F2212353EE4906578F2
:1012C300F0300912122FC5906331EFF0D394004030
:1012D30005E0FF12484E200803021459122E3E90D7
:1012E3006331EFF070030211F0906375E054BF2493
:1012F3007F70030213C214700302139A2402600363
:101303000213FB200B077E1B7F2912353E200F03A0
:1013130002145990634DE07006906351E06067904A
:101323006682E0FF90634DE0B50724906683E0FE9C
:1013330090634EE0B50618906684E0FE90634FE03C
:10134300B5060C906685E0FE906350E06E603790C2
:101353006351E06F6003021459906683E0FF90636A
:1013630052E06F6003021459906684E0FF90635368
:10137300E06F6003021459906685E0FF906354E0C8
:101383006F6003021459C2039065777401F0124829
:1013930051750A0102145990668BE060037401F0E1
:1013A30090667AE0FF906377E06F600302145990D0
:1013B300667AE004F0E4F50A906575F0021459309A
:1013C3000303021459906344E070030211F0906325
:1013D30055740AF012001ED203E4F50A906575F005
:1013E30090668604F0E4906679F0A3F0200B677EA4
:1013F3001B7F3712353E805E90668BE0600374017D
:10140300F0300352906375E020E74B906377E0FF81
:10141300906679E0FE6F600D906681E07007EE14D0
:101423006F70338013906679E004F0906331E0FFCE
:10143300D3940440031248509060007482F0A37464
:1014430001F0906377E0906002F07E607F007D039F
:10145300123EAD0211F0200303021571E50A706814
:10146300123D0CEF60237E647F75906476E0240464
:10147300FD123EAD906681E07009906355E0F50A78
:101483000211F0E4F50A0211F0906686E0D3943C71
:101493004036906681E0703090668604F012484FC3
:1014A300E4906475F0A37412F090667AE090647728
:1014B300F0A374FDF090610563A20190647963A2C7
:1014C300017F121229B2809E12484A8F24E524B468
:1014D30001159060007483F0E4A3F07E607F007DCB
:1014E30002123EAD0211F0E524D39401401C90603A
:1014F300007483F0A37401F0E52424FEA3F07E605E
:101503007F007D03123EAD0211F0E50A6401600322
:101513000211F0906575E004F0200B077E1B7F41FC
:1015230012353E906355E0C394C85004E02432F072
:10153300906575E0C39405400DC203E4906577F0B0
:101543001248510211F07C667D82906349E0FAA350
:10155300E0FB7F0212403E7E647F75906476E02458
:1015630004FD123EAD906355E0F50A0211F0E50A61
:10157300640160030211F0906577E014604624FE75
:101583006042147003021664240460030211F0E441
:10159300F50C200F139065777404F0906575E05493
:1015A30001F0750A010211F09080027410F0E490CA
:1015B3006577F090657504F0750AFA90668274FF9A
:1015C300F00211F0906682E0700302164E9064758B
:1015D3007480F09064777401F0E4A3F0A304F0A3A3
:1015E3007430F0A3747BF0E4F524747C2524F58235
:1015F300E43464F583747DF0747D2524F582E4344A
:1016030064F583E4F0E5242407906476F07C667D3A
:1016130082906349E0FAA3E0FB7F0212403E7E64BE
:101623007F75E5242409FD123EAD906681E0601BC1
:1016330012001ED203E4F50A906575F090668604E5
:10164300F0E4906679F0A3F00211F0300F07E49014
:101653006577F080069065777404F0750AFA0211D5
:10166300F09080027410F0750A05906575E06401CE
:10167300FFF09065777401F0EF7019906351E060AB
:1016830013FCA3E0FDA3E0FEA3E0FF906682120F2C
:10169300150211F090634DE0FCA3E0FDA3E0FEA36F
:0D16A300E0FF906682120F150211F080FE2C
:0116B0002217
:10002600906376E0B444047F0180027F009063759C
:10003600E0B447047E0180027E00EE5F604A906372
:100046003EE0906377F090633FE0906378F09063D2
:1000560040E0906379F0906341E090637AF09063BA
:1000660042E090637BF0906343E090637CF09063A2
:10007600767452F09062AE63A2019080A863A201EA
:100086007F061229B2020849906331E0C3940850F2
:100096000302085290633EE0FF906377E06F6003CF
:1000A60002085290633FE0FF906378E06F600302BE
:1000B6000852906340E0FF906379E06F60030208A6
:1000C60052906341E0FF90637AE06F60030208524A
:1000D600906342E0FF90637BE06F600302085290FA
:1000E6006343E0FF90637CE06F6003020852906315
:1000F60076E0B444159062AEE0B4FF0E63A20190C0
:1001060080A863A2017F061229B290668BE0600385
:100116007401F090668C7464F09063767452F0907B
:100126006375E0646D60030202537BFF7A1B794CB2
:100136001217137BFF7A1B796690633EE0F52DA3B9
:10014600E0F52EA3E0F52FA3E0F530A3E0F531A30B
:10015600E0F532121713752DFF752E1B752FC3751B
:1001660030FF75311B7532CF7BFF7A1B799C1217D6
:10017600137BFF7A1B79D81217137BFF7A1C793E03
:100186001217137BFF7A1C796B906344E0F52DA35D
:10019600E0F52EA3E0F52FA3E0F5301217137BFF51
:1001A6007A1C799590634DE0F52DA3E0F52EA3E03A
:1001B600F52FA3E0F5301217137BFF7A1C79C39055
:1001C6006351E0F52DA3E0F52EA3E0F52FA3E0F5AE
:1001D600301217137BFF7A1C79F190633AE0F52D04
:1001E600A3E0F52EA3E0F52FA3E0F5301217137B5D
:1001F600FF7A1D7914906336E0F52DA3E0F52EA362
:10020600E0F52FA3E0F5301217137BFF7A1D793145
:100216001217137BFF7A1D795AA20FE433F52D12BC
:1002260017137BFF7A1D798A906681E0F52D1217E8
:10023600137BFF7A1D79B590668BE0F52D121713A7
:100246001226CC7BFF7A1D79E8121713229063756C
:10025600E0644C70737E1D7FEEFBFDFC1232439012
:10026600637DE0F525A3E0F526E4F528E525906312
:100276007FF0A3E526F07E1E7F297C637D7F7B02CF
:10028600123243E4F527852682852583E0FF747FB5
:100296002527F582E43463F583EFF00526E526701D
:1002A6000205250527E527B410DC7E1E7F2C7C631E
:1002B6007D7F7B101232430528E528C3941040AC9D
:1002C6007E1E7F2F12353E22906375E0646C70604F
:1002D600F5297E1E7F31FBFDFC123243E4F528E44E
:1002E60090637FF0A3E529F07E1E7F297C637D7FE6
:1002F6007B02123243E4F527A829E6FF747F2527FF
:10030600F582E43463F583EFF005290527E527B484
:1003160010E67E1E7F2C7C637D7F7B1012324305A8
:1003260028E528C3940840B77E1E7F2F12353E224B
:10033600906375E0644B7061F52774672527F58235
:10034600E43463F583E0603274672527F582E4348C
:1003560063F583E0F4602374672527F582E434634C
:10036600F583E0FF747D2527F582E43463F583E0A9
:10037600B507100527E527B408C09061047432F06C
:100386000208499063757421F0300B030208497E18
:100396001E7F6C12353E020849906375E0B4521A0E
:1003A600200B077E1E7F7412353E9063757472F0C3
:1003B6007E637F757D08123E2622906375E0644950
:1003C6007045200B077E1E7F7F12353E90637DE0D1
:1003D600F525A3E0F526E4F527852682852583E025
:1003E600FF747F2527F582E43463F583EFF0052655
:1003F600E526700205250527E527B480DC7E637FA8
:10040600757D8A123E2622906375E064437046200D
:100416000B077E1E7F8712353E90637DE0F525A390
:10042600E0F526E4F527852682852583E493FF7487
:100436007F2527F582E43463F583EFF00526E5266C
:10044600700205250527E527B480DB7E637F757D71
:100456008A123E2622906375E0645A7053200B0779
:100466007E1E7F9012353E90637DE0F525A3E0F574
:10047600267C637D7F7B80AF26AE251246E2E4F5BF
:1004860027852682852583E493FF747F2527F582B9
:10049600E43463F583EFF00526E5267002052505AD
:1004A60027E527B480DB7E637F757D8A123E262290
:1004B600906375E06444600302054790637DE0FF46
:1004C60064447003020849EFB4310CC20B7E1E7FF0
:1004D6009C12353E02084990637DE0B4300CD20B85
:1004E6007E1E7FA812353E02084990637DE0B43235
:1004F6000CD20C7E1E7FB512353E02084990637DF4
:10050600E0B4330CC20C7E1E7FC312353E0208498E
:1005160090637DE0B4340CD20D7E1E7FD212353E40
:1005260002084990637DE0B4350CC20D7E1E7FDF64
:1005360012353E02084990637DE0FF12484D0208DD
:1005460049906104E07013200B077E1E7FED123583
:100556003E9063757421F00208499061047432F08C
:10056600906375E0FFB45104C2AF80FEEF6457702C
:1005760045200B077E1E7FFB12353E90637EE09082
:100586006331F0E4F527906331E0FFE527C39F4030
:1005960003020849747F2527F582E43463F583E076
:1005A600FF90637DE0252724ADF582E43461F58371
:1005B600EFF0052780D0906375E064536003020670
:1005C6006A200B077E1F7F0612353E90633EE0FFD2
:1005D6009061B6E06F703C90633FE0FF9061B7E0DA
:1005E6006F7030906340E0FF9061B8E0B5072490EB
:1005F6006341E0FF9061B9E0B50718906342E0FF00
:100606009061BAE0B5070C906343E0FF9061BBE0F0
:100616006F60169063757421F0300B030208497EF3
:100626001F7F1512353E020849E4F527E4F50DAFA4
:1006360027FE74AD2527F582E43461F583E0FD12CB
:10064600473C0527E527C394FE40E1C2AFE4907F0F
:10065600F0F0A3F0907FFD74AAF0A374FFF0A374EA
:1006660055F080FE906375E0644F704C90637DE0BA
:10067600F525A3E0F526E5264525700A200B077E1D
:100686001F7F1E12353E200B077E1F7F2512353E2B
:10069600E4F527747F2527F582E43463F583E08546
:1006A6002682852583F00526E52670020525052781
:1006B600E527B480DE020849906375E0FFB4452162
:1006C60090637DE0FDA3E0907FF0CDF0A3EDF0C256
:1006D600AF907FFD74AAF0A374FFF0A37455F08069
:1006E600FEEF6465600302085290637DE0FFA3E0BD
:1006F600907FF0CFF0A3EFF0E4F525F526D3907FB9
:10070600F1E09526907FF0E095254020E4F50D2553
:1007160026FFE5253401FE852682852583E0FD1228
:10072600473C0526E5267002052580D17E1F7F27DA
:10073600123F34EF4E6020120003906344EFF01234
:100746000003906345EFF0120003906346EFF0124A
:100756000003906347EFF07E1F7F2D123F34EF4E6C
:10076600602012000390634DEFF012000390634E79
:10077600EFF012000390634FEFF012000390635006
:10078600EFF07E1F7F33123F34EF4E6020120003DE
:10079600906351EFF0120003906352EFF0120003E2
:1007A600906353EFF0120003906354EFF07E1F7FC7
:1007B60039123F34EF4E602012000390633AEFF097
:1007C60012000390633BEFF012000390633CEFF0DE
:1007D60012000390633DEFF07E1F7F3F123F34EF20
:1007E6004E6020120003906336EFF0120003906310
:1007F60037EFF0120003906338EFF01200039063B6
:1008060039EFF0E4F527E4F50DE5272401FFE4339D
:10081600FE74362527F582E43463F583E0FD12473E
:100826003C0527E527C3944340DCC2AFE4907FF044
:10083600F0A3F0907FFD74AAF0A374FFF0A37455A3
:0C084600F080FE7E637F757D08123E2668
:010852002283
:1046AA00AE07EEC39430400BEED394395005EE2496
:1046BA00D0FF22EEC39461400BEED394665005EE10
:1046CA0024A9FF22EEC39441400BEED39446500531
:0846DA00EE24C9FF22AF062205
:1047FE009062ADE004F070069062ACE004F090625E
:0A480E00ACE0FEA3E0FF1247A82271
:100003001247FE1246AAEFC454F0FEC0061247FE82
:080013001246AAD0E02FFF22E3
:10450D00E4906BD4F01247FE906BD5EFF0C394306E
:10451D004018E0FFD394395011906BD4E02405F589
:10452D0082E43461F583EFF08011906BD4E02405C3
:10453D00F582E43461F583E4F0800C906BD4E004F3
:10454D00F0E0D3940840BE752900752A00752B0044
:0C455D00E4F52C7B017A617905122C9AA0
:01456900222F
:043F34008E2A8F2B17
:103F38009062ACE4F0A374FFF01247FEEF606EF4F9
:103F4800606B852B82852A83E493B507EC752C0179
:103F5800E52B252CF582E4352AF583E4936025903A
:103F680062ADE0252CFF9062ACE03400FE1247A859
:103F7800E52B252CF582E4352AF583E493B507046F
:103F8800052C80CCE52B252CF582E4352AF583E435
:103F98009370A6E52C24FFFFE434FFFE9062ADE0A9
:103FA8002FF09062ACE03EF07E007F0122E4FEFF3D
:013FB80022E6
:1039A4007E1F7F45123F34EF4E70037F01227E1F3E
:1039B4007F48123F34EF4E600C1247FEEF24D024B0
:1039C400FF920F8002D20F7E1F7F4E123F34EF4EC4
:1039D400600C1247FEEF24D0906681F08005E490DD
:1039E4006681F07E1F7F54123F34EF4E600C124705
:1039F400FEEF24D090668BF08005E490668BF07E19
:103A04001F7F5A123F34EF4E600C1247FEEF24D052
:103A140024FF92018002C20190633E63A20190667A
:103A24007B63A2017F061229B230013B7E1F7F60B7
:103A3400123F34EF4E603012000390667BEFF012B9
:103A4400000390667CEFF012000390667DEFF012A5
:103A5400000390667EEFF012000390667FEFF01291
:0A3A64000003906680EFF07F00225F
:10461F00906576E0C3947C503D906576E0FE04F0A3
:10462F0074B42EF582E43462F583EFF0BF0A27905D
:10463F006576E0FF04F074B42FF582E43462F583FD
:10464F00E4F0906576E0FF123FB99065767408F05C
:07465F009062B5E004F022B7
:1045C6009080007480F090633663A201F583F582D3
:1045D60063A2017F081229B290633E63A201908014
:1045E6008863A2017F0A1229B2908092E4F0A37434
:1045F60032F0A37401F0906348E0FF9080B1F09030
:1046060080E1EFF09080957455F0A3F090800074EF
:0946160001F090800974F0F0221B
:10414000908009E04410F09080A0E0706C9080A115
:104150007482F09080A874FFF0A3F0A3F0A3F07F26
:10416000039080AEEFF07FCBA3EFF07F039080ACA5
:10417000EFF0A374CBF09080007402F0906BC81243
:104180000F2100000000906BC8E0908040F0906B21
:10419000C9E0908041F0906BCAE0908042F0906B53
:1041A000CBE0908043F0A3E4F0A3F0A3F0A3F09061
:0941B0008018F0A3F0A3F0A3F0C5
:0141B90022E3
:10456A00908009E04440F09080D17482F07F0390FB
:10457A0080DEEFF0A374CCF09080027402F0906BAE
:10458A00CC120F2100000000906BCCE0908058F014
:10459A00906BCDE0908059F0906BCEE090805AF00D
:1045AA00906BCFE090805BF0A3E4F0A3F0A3F0A3BC
:0B45BA00F0908030F0A3F0A3F0A3F01D
:0145C50022D3
:1041BA00908009E04420F09080B8E0706C9080B95B
:1041CA007482F07F039080C6EFF07FCDA3EFF07F7B
:1041DA00039080C4EFF0A374CDF09080C074FFF018
:1041EA00A3F0A3F0A3F09080017402F0906BD012B8
:1041FA000F2100000000906BD0E090804CF0906B93
:10420A00D1E090804DF0906BD2E090804EF0906BB0
:10421A00D3E090804FF0A3E4F0A3F0A3F0A3F090D2
:09422A008024F0A3F0A3F0A3F03E
:014233002268
:10403E008C258D26A907EAFDE975F018A424ACFF9E
:10404E00E5F034808F82F583EDF0EBFDE975F01825
:10405E00A4FFAEF024ACFBEE34808B82F583A3ED8F
:10406E00F08526828C83E0FDEF24A8FFEE3480FEDF
:10407E008F82F583EDF08526828C83A3E08F828E6E
:10408E0083A3F0852682852583A3A3E0FDE975F041
:10409E0018A424A8FFE5F03480FE8F82F583A3A335
:1040AE00EDF08526828C83A3A3A3E08F828E83A35B
:0440BE00A3A3F022A6
:063E26008D2AAB07AA067D
:103E2C00908000E030E5079065787401F022906B8B
:103E3C00C8E0FCA3E0FDA3E0FEA3E0F52E8E2D8DE3
:103E4C002C8C2BAE02AF038E838F8263A201E52DE7
:103E5C00540744C0F583852E8263A201AF2A122A2F
:103E6C0024E4FCFDFEE52E252AF52EEE352DF52D50
:103E7C00ED352CF52CEC352BF52B908040E52BF00B
:103E8C00A3E52CF0A3E52DF0A3E52EF090800074B3
:103E9C0020F0AF2EAE2DAD2CAC2B906BC8120F15A5
:013EAC0022F3
:063EAD008D25AB07AA06FB
:103EB300908002E030E5079065787403F022906B00
:103EC300CCE0FCA3E0FDA3E0FEA3E0F5298E288D62
:103ED300278C26AE02AF038E838F8263A201E5286F
:103EE300540744D0F58385298263A201AF25122AA2
:103EF30024E4FCFDFEE5292525F529EE3528F528E2
:103F0300ED3527F527EC3526F526908058E526F084
:103F1300A3E527F0A3E528F0A3E529F09080027438
:103F230020F0AF29AE28AD27AC26906BCC120F152D
:013F3300226B
:023A6E008F25A2
:103A7000908001E030E5099065787402F07F0022C3
:103A8000906BD0E0FCA3E0FDA3E0FEA3E0F5298E5F
:103A9000288D278C2690667B63A201E52854074475
:103AA000C8F58385298263A2017F06122A3AE52997
:103AB0002406F529E43528F528E43527F527E435EB
:103AC00026F52690657963A201E528540744C8F5D8
:103AD0008385298263A201AF25122A3AE4FCFDFE08
:103AE000E5292525F529EE3528F528ED3527F52793
:103AF000EC3526F52690804CE526F0A3E527F0A3CB
:103B0000E528F0A3E529F09080017420F0AF29AEFC
:0D3B100028AD27AC26906BD0120F15AF2505
:013B1D002285
:10334A009081E0E0F52505250525052505250525B6
:10335A0005250525052505250525908010E0F52874
:10336A00A3E0F529A3E0F52AA3E0F52B9081E1E09B
:10337A00F525052505250525052505250525052503
:10338A00052505250525908014E0F52CA3E0F52DEB
:10339A00A3E0F52EA3E0F52FE52EB52A08E52FB513
:1033AA002B037F0022E4F525E52E540744E0F5833C
:1033BA00852F8263A20190637563A2017F08122A96
:1033CA006A90637763A2019062AE63A2017F0612DC
:1033DA0029B2906375E0F526A3E0F527E4F5259078
:1033EA006375E0702AA3E024F8F525E52E54074416
:1033FA00E0F583852F8274082582F582E43583F50A
:10340A008363A20190637563A201AF25122A6AAE93
:10341A0026E4FCFDE52F2527F52FE52E3EF52EEDBA
:10342A00352DF52DEC352CF52C908014E52CF0A3D8
:10343A00E52DF0A3E52EF0A3E52FF090800074406F
:03344A00F0AF25BB
:01344D00225C
:102E3E009081E6E0F52505250525052505250525C1
:102E4E0005250525052505250525908028E0F5286D
:102E5E00A3E0F529A3E0F52AA3E0F52B9081E7E0A6
:102E6E00F525052505250525052505250525052514
:102E7E0005250525052590802CE0F52CA3E0F52DE4
:102E8E00A3E0F52EA3E0F52FE4F525E52EB52A0AED
:102E9E00E52FB52B05C208022FAAE52E540744F0E4
:102EAE00F583852F8263A20190637563A2017F086B
:102EBE00122A6A906375E0F526A3E0F527E527450B
:102ECE002670099080027410F07F0022906682E0D6
:102EDE00FFF46030906377E06F6003022F719066AD
:102EEE0083E0FF906378E06F7079906684E0FF90E6
:102EFE006379E06F706D906685E0FF90637AE06FA6
:102F0E006031805F906377E0906682F0906378E046
:102F1E00906683F0906379E0906684F090637AE037
:102F2E00906685F090637BE0FFA3E0906349CFF05D
:102F3E00A3EFF0906375E0702AA3E024F8F525E581
:102F4E002E540744F0F583852F8274082582F5826E
:102F5E00E43583F58363A20190637563A201AF2507
:102F6E00122A6AAE26E4FCFDE52F2527F52FE52E65
:102F7E003EF52EED352DF52DEC352CF52CAF2BAE7B
:102F8E002AAD29AC28AB2FAA2EA92DA82CD3120F0F
:102F9E000440099080027410F07F002290802CE58E
:102FAE002CF0A3E52DF0A3E52EF0A3E52FF09080F5
:062FBE00027440F0AF2593
:012FC40022EA
:102FC5009081E3E0F525052505250525052505253C
:102FD5000525052505250525052590801CE0F528F1
:102FE500A3E0F529A3E0F52AA3E0F52B9081E4E021
:102FF500F52505250525052505250525052505258C
:10300500052505250525908020E0F52CA3E0F52D67
:10301500A3E0F52EA3E0F52FE4F525E52EB52A0A64
:10302500E52FB52B05C20902311BE52E540744E8EF
:10303500F583852F8263A20190600463A2017F0E50
:10304500122A80906004E0F526A3E0F52790600C35
:10305500E0FFF4604A90667BE0FEEF6E7079A3E0D6
:10306500FF90600DE06F706F90667DE0FF90600EE1
:10307500E06F706390667EE0FF90600FE06F7057C1
:1030850090667FE0FF906010E06F704B906680E087
:10309500FF906011E06F703FE4906013F08008903E
:1030A500601374FFF0D2D9906004E0702AA3E02485
:1030B500F2F525E52E540744E8F583852F82740E35
:1030C5002582F582E43583F58363A201906004636C
:1030D500A201AF25122A80AE26E4FCFDE52F2527A7
:1030E500F52FE52E3EF52EED352DF52DEC352CF590
:1030F5002CAF2BAE2AAD29AC28AB2FAA2EA92DA813
:103105002CD3120F045006E527452670099080013F
:103115007410F07F0022908020E52CF0A3E52DF0BF
:10312500A3E52EF0A3E52FF09080017440F0AF25C4
:013135002277
:04353E008E2A8F2B17
:10354200908000E030E5079065787401F022906B7E
:10355200C8E0FCA3E0FDA3E0FEA3E0F5318E308DD0
:103562002F8C2EE531FFE5305407FEE42FF52DEECA
:1035720034C0F52C852D82F5837423F0052DE52DBD
:103582007002052C532CC7F582852C83740AF00532
:103592002DE52D7002052C532CC790633E63A201CA
:1035A200852C83852D8263A2017F06122A2474064C
:1035B200252DF52DE4352CF52C852A83852B826368
:1035C200A201852C83852D8263A201122A08E4FCC4
:1035D200FDFE906BC8E0F8A3E0F9A3E0FAA3E02FA8
:1035E200FFEE3AFEED39FDEC38FCEF2408FFE43E35
:1035F200FEE43DFDE43CFC906BC8120F15906BC8D5
:10360200E0908040F0906BC9E0908041F0906BCAEE
:10361200E0908042F0906BCBE0908043F09080008D
:033622007420F021
:013625002282
:0A3243008E2A8F2B8C2C8D2D8B2EE4
:10324D00908000E030E5079065787401F022906B76
:10325D00C8E0FCA3E0FDA3E0FEA3E0F5348E338DC2
:10326D00328C31E534FFE5335407FEE42FF530EEB3
:10327D0034C0F52F853082F5837423F00530E530A9
:10328D007002052F532FC7F582852F83740AF00521
:10329D0030E5307002052F532FC790633E63A201B6
:1032AD00852F8385308263A2017F06122A2474063E
:1032BD002530F530E4352FF52F852A83852B826354
:1032CD00A201852F8385308263A201122A088F35D2
:1032DD00EF2530F530E4352FF52FE52E6017852CD1
:1032ED0083852D8263A201852F8385308263A201A0
:1032FD00AF2E122A24E5352408252EF52EFFE4FCE9
:10330D00FDFEE5342FF534EE3533F533ED3532F57D
:10331D0032EC3531F531908040E531F0A3E532F0F6
:10332D00A3E533F0A3E534F09080007420F0AF34C2
:0C333D00AE33AD32AC31906BC8120F15EE
:013349002261
:0638C9008E268F278D28DA
:1038CF00908000E030E5079065787401F022906BEE
:1038DF00C8E0FCA3E0FDA3E0FEA3E0F52E8E2D8D46
:1038EF002C8C2BE52EFFE52D5407FEE42FF52AEE49
:1038FF0034C0F529852A82F5837423F0052AE52A39
:10390F00700205295329C7F582852983EBF0052A13
:10391F00E52A700205295329C790633E63A20185EA
:10392F002983852A8263A2017F06122A2474062521
:10393F002AF52AE43529F52985268385278263A26E
:10394F0001852983852A8263A201AF28122A247454
:10395F00082528F528FFE4FCFDFEE52E2FF52EEEB9
:10396F00352DF52DED352CF52CEC352BF52B9080D9
:10397F0040E52BF0A3E52CF0A3E52DF0A3E52EF009
:10398F009080007420F0AF2EAE2DAD2CAC2B906B31
:04399F00C8120F1526
:0139A3002201
:023FB9008F4631
:103FBB00908000E030E5079065787401F022906BFB
:103FCB00C8E0FCA3E0FDA3E0FEA3E0F54A8E498D1B
:103FDB00488C47E54AFFE5495407FEE42FFFEE34D2
:103FEB00C09062B463A201F5838F8263A201AF46D6
:103FFB00122A24E4FCFDFEE54A2546F54AEE354936
:10400B00F549ED3548F548EC3547F547908040E5E7
:10401B0047F0A3E548F0A3E549F0A3E54AF090800B
:10402B00007420F0AF4AAE49AD48AC47906BC81254
:02403B000F155F
:01403D002260
:06370C008E288F29AB0599
:10371200908000E030E5079065787401F022906BAC
:10372200C8E0FCA3E0FDA3E0FEA3E0F52F8E2E8D02
:103732002D8C2CE52FFFE52E5407FEE42FF52BEE02
:1037420034C0F52A852B82F5837423F0052BE52BF3
:103752007002052A532AC7F582852A83EBF0052BCE
:10376200E52B7002052A90633E63A201852A8385B8
:103772002B8263A2017F06122A247406252BF52BC5
:10378200E4352AF52A532AC7E528852B82852A8320
:10379200F0052BE52B7002052A532AC7F582852AEC
:1037A20083E529F0052BE52B7002052A532AC7E58C
:1037B2002F240AF52FE4352EF52EE4352DF52DE4D0
:1037C200352CF52C908040E52CF0A3E52DF0A3E5F7
:1037D2002EF0A3E52FF09080007420F0AF2FAE2ED4
:0A37E200AD2DAC2C906BC8120F1532
:0137EC0022BA
:10444A00908009E04480F09080E97401F07F09903F
:10445A0080F6EFF0A37464F09080037402F0908009
:10446A0000E020E1F9906AC4120F210000000090D8
:10447A006AC4E0908064F0906AC5E0908065F0902C
:10448A006AC6E0908066F0906AC7E0908067F0A301
:10449A00E4F0A3F0A3F0A3F090803CF0A3F0A3F023
:0244AA00A3F07D
:0144AC0022ED
:1037ED009081E9E0F5260526052605260526052600
:1037FD0005260526052605260526908034E0F527A5
:10380D00A3E0F528A3E0F529A3E0F52A9081EAE0ED
:10381D00F526052605260526052605260526052653
:10382D00052605260526908038E0F52BA3E0F52C1E
:10383D00A3E0F52DA3E0F52EE52DB52908E52EB570
:10384D002A037F0022AF2EAE2DAD2CAC2BAB2AAAB6
:10385D0029A928A827D3120F04400AAF2EAE2AEEAD
:10386D009FF526800AAF2EEFF404AE2A2EF526E53D
:10387D002D540744E0F583852E8263A201906AC81A
:10388D0063A201AF26122A98E4FCFDFEE52E252643
:10389D00F52EEE352DF52DED352CF52CEC352BF5D6
:1038AD002B908038E52BF0A3E52CF0A3E52DF0A3AC
:0B38BD00E52EF09080037440F0AF2671
:0138C80022DD
:02344E008F26C7
:103450009080E8E0640660037FFF22906AC4E0FC8D
:10346000A3E0FDA3E0FEA3E0F52A8E298D288C279A
:10347000E4FFFEFDFCAB2AAA29A928A827C3120F46
:103480000470609081F9E0F527906AC4E0FCA3E045
:10349000FDA3E0FEA3E0FFE4FAF9F8EF2401FFEA60
:1034A0003EFEE93DFDE83CFC906AC4120F15906AAF
:1034B000C4E0FCA3E0FDA3E0FEA3E0FFE4F8EF24FA
:1034C00001FFEA3EFEE93DFDE83CFC906AC4120FB4
:1034D00015908064E0F527A3E0F528A3E0F529A383
:1034E000E0F52A906AC863A201E529540744D8F59B
:1034F00083852A8263A201AF26122A52E4FCFDFED4
:10350000E52A2526F52AEE3529F529ED3528F52871
:10351000EC3527F527908064E527F0A3E528F0A394
:10352000E529F0A3E52AF09080037420F0AF2AAEDD
:0D35300029AD28AC27906AC4120F157F004A
:01353D00226B
:1047A800A2AF9210C2AF438E2075D2028F828E8341
:0C47B800E0FFE4F5D2538EDFA21092AFB8
:0147C40022D2
:10473C00E5D220E0FBA2AF9210C2AF43D2028F822F
:10474C008E83EDF075D25063D250A21092AFE5D2A9
:03475C0020E0FB5F
:01475F002237
:1040C200E4FDED2401FFE433FE1247A874362DF51A
:1040D20082E43463F583EFF00DBD3FE6E4FDED24A9
:1040E2007FFFE433FE1247A8742D2DF582E434617C
:1040F200F583EFF0742D2DF582E43461F583E070E1
:104102001B742D2DF582E43461F5837420F0742E36
:104112002DF582E43461F583E4F080040DBD80BEA8
:10412200E49061ACF0FDEDFF7E001247A874AD2D66
:0D413200F582E43461F583EFF00DBDFEE988
:01413F00225D
:0246E2008B2A21
:1046E400A2AF9210C2AF85A22B53A2FE8E838F82FB
:1046F40005A28C838D827409122AAEE52A53A2FE88
:1047040043A220122AB053A2DF852BA2A21092AF9B
:01471400FFA5
:014715002281
:1047C500A2AF9210C2AF8C838D82EF122AAE43A2A4
:0C47D50020122AB053A2DFA21092AFFF06
:0147E10022B5
:024760008F25A3
:10476200A2AF9210C2AFE4F5838D827406122AAE14
:10477200E52543A220122AB053A2DFA21092AF7FF6
:014782000135
:014783002213
:024784008F257F
:10478600A2AF9210C2AFE4F5838D82740A122AAEEC
:10479600E52543A220122AB053A2DFA21092AF7FD2
:0147A6000111
:0147A70022EF
:1028D700A907E7FFA805EF93C3966008403B74FC80
:1028E7002FFF80F00F08EF93C3966008402B74FB0F
:1028F7002FFF80E00F08EF93C3966008401B74FA20
:102907002FFF80D00F08EF93D3966008400B74F920
:102917002FFF80C01F1F1F1F1FEF54FEF80303F771
:10292700E893FC08E893FD08E893FE08E893FF2284
:1029370009E993C39D6008402974FB29F980F109CF
:10294700E993C39E6008401A74FA29F980E209E9FD
:1029570093D39F6008400B74F929F980D31919198B
:102967001919E9C313C313FF22740093F8ECC39832
:102977004024701F740193F8EDC3984019701474C4
:0E2987000293F8EEC398400E7009740393F8A3
:10299500EFC39840037F00227F0122EDF8E6F0089F
:1029A500A3DFFA22EDF8E0F608A3DFFA22E0A3633D
:1029B500A201F0A363A201DFF475A2002263A201C4
:1029C500F0A363A20122E0A363A201F0A363A20125
:1029D500E0A363A201F0A363A201E463A201F0A353
:1029E50063A201DFE175A20022E0A363A2016DFEEF
:1029F500936CFDEE058393FC158363A201DFEA75F5
:102A0500A200227F00E493A363A201F00F600CA350
:102A1500E583C2E3F58363A20180EA75A20022E0A3
:102A2500A363A201F0A3E583C2E3F58363A201DFFB
:102A3500EE75A20022E0A363A201F0A3E583C2E440
:102A4500D2E3F58363A201DFEC75A20022E0A36364
:102A5500A201F0A3E58344F8C2E5F58363A201DF93
:102A6500EC75A20022E583C2E3F583E0A363A2012E
:102A7500F0A363A201DFEE75A20022E583C2E4D2D2
:0A2A8500E3F583E0A363A201F0A3D0
:102A8F0063A201DFEC75A20022E58344F8F583E031
:102A9F00A363A201F0A363A201DFEE75A20022F9E6
:102AAF0022C002C004C00612FFF0D006D004D0022C
:012ABF0022F4
:10233E003E2A2C312CCFE0F0E0ECE5F2F0FB20F859
:10234E00E8EDFB2043414E0A003E4C2C6B30312C05
:10235E0025732C43EAEEF0EEF1F2FC20EDE020F8CE
:10236E00E8EDE52043414E2C30202D20353030EA6B
:10237E00E1283530EC292C31202D203530EAE128AA
:10238E00353030EC290A0030202D20353030EAE18E
:10239E00283530EC290031202D203530EAE1283562
:1023AE003030EC29003E2A2C312CCFE0F0E0ECE569
:1023BE00F2F0FB20EFF0EEF2EEEAEEEBE020C2EEF2
:1023CE00E4EEEBE5E90A003E4C2C4930312C256C4D
:1023DE00752CD1EAEEF0EEF1F2FC20EEE1ECE5ED3B
:1023EE00E02C343830302C393630302C3139323014
:1023FE00300A003E532C4931322C2562752CC0E434
:10240E00F0E5F120E1EBEEEAE020D2C8D220EDE0DB
:10241E0020F8E8EDE50A003E532C4931332C2562B5
:10242E00752CC0E4F0E5F120EFF0E8E1EEF0E00A03
:10243E00003E532C5630392C25752CD6E8EAEB206D
:10244E00EEEFF0EEF1E020EFF0E8E1EEF0E0202824
:10245E00F1290A003E532C6630302C25662CCCE038
:10246E00F1F8F2E0E120D2310A003E532C66303111
:10247E002C25662CCCE0F1F8F2E0E120D2320A00F5
:10248E003E532C6630322C25662CCCE0F1F8F2E06F
:10249E00E120D2330A003E532C6630332C25662CB5
:1024AE00CCE0F1F8F2E0E120D2340A003E532C6683
:1024BE0030342C25662CCCE0F1F8F2E0E1204731E7
:1024CE000A003E532C6630352C25662CCCE0F1F8F4
:1024DE00F2E0E12047320A003E532C6630362C25BE
:1024EE00662CCCE0F1F8F2E0E12047330A003E53CF
:1024FE002C6630372C25662CCCE0F1F8F2E0E1208A
:10250E0047340A003E532C6630382C25662CCCE01E
:10251E00F1F8F2E0E12050310A003E532C663039DA
:10252E002C25662CCCE0F1F8F2E0E12050320A00C6
:10253E003E532C6631302C25662CCCE0F1F8F2E0BF
:10254E00E12050330A003E532C6631312C25662C87
:10255E00CCE0F1F8F2E0E12050340A003C6B30316F
:10256E003D003C4930313D003C4931323D003C5646
:10257E0030383D003C5630393D003C4931333D004A
:10258E002043616E457247495400200A0020436182
:10259E006E457272434821000A000AC7E0EFF0EE62
:1025AE00F13A00496E69745443500A004C697374D1
:1025BE00656E5443500A00534F434B5F5443505F74
:1025CE0045535441424C49534845440A000A2D3E56
:1025DE0020000A3C2D20000ACEF2E2E5F23A00CEAF
:1025EE00F8E8E1EAE02021000A56616C3A0025661F
:1025FE0000202566202A202566203D202020202030
:10260E0020202020202020202020202020202020BC
:10261E0020202020002025352E306620202020204E
:10262E00202020202020202020202020202020209C
:10263E0020202020202020202020202020003C664A
:10264E0030303D0000003C6630313D0000003C66FD
:10265E0030323D0000003C6630333D0000003C66E9
:10266E0030343D0000003C6630353D0000003C66D5
:10267E0030363D0000003C6630373D0000003C66C1
:10268E0030383D0000003C6630393D0000003C66AD
:10269E0031303D0000003C6631313D0000003C66AB
:1026AE0031323D0000003C6631333D0000003C6697
:0E26BE0031343D0000003C6631353D00000027
:1047E80052668D000000000000000000000000007C
:0547F8000000000000BC
:01484D002248
:030023000243177E
:10431700C0E0C083C082C0D075D01830982CE55D4E
:1043270025E9F5EB30D709E55C25F904F5FB8006AF
:10433700E55C25F9F5FBD291749C2562F582E4349E
:1043470069F583E599F00562C298309922E563C360
:1043570095615013AF630563749C2FF582E4346A4B
:10436700F583E0F5998006C219D296C290C299D01A
:08437700D0D082D083D0E032E7
:10471600C2A9438902758C48758A4875D90475DB28
:104726004875DC4875DD4875DE48E4F5E9F5F9C2FB
:06473600D9D28CD2DE2274
:1026CC007BFF7A23793E12171390689FE070147584
:1026DC002DFF752E23752F957BFF7A2379571217B3
:1026EC00138012752DFF752E23752FA47BFF7A2373
:1026FC0079571217137BFF7A2379B3121713906A49
:10270C00C2E0FEA3E0FFC3E49FFFE49EFEAB07FA2A
:10271C003395E0F9F87F007E8C7D0A7C00120E6404
:10272C008F308E2F8D2E8C2D7BFF7A2379D512171F
:10273C00137BFF7A2479019068A0E0F52D12171312
:10274C007BFF7A247925906928E0F52D1217137BED
:10275C00FF7A24793F9068A3E0F52DA3E0F52E12C3
:10276C0017137BFF7A24796290696CE0FCA3E0FD7F
:10277C00A3E0FEA3E0F5308E2F8D2E8C2D121713B7
:10278C007BFF7A247978906970E0FCA3E0FDA3E0EC
:10279C00FEA3E0F5308E2F8D2E8C2D1217137BFFA0
:1027AC007A24798E906974E0FCA3E0FDA3E0FEA38B
:1027BC00E0F5308E2F8D2E8C2D1217137BFF7A2483
:1027CC0079A4906978E0FCA3E0FDA3E0FEA3E0F51A
:1027DC00308E2F8D2E8C2D1217137BFF7A2479BA05
:1027EC0090697CE0FCA3E0FDA3E0FEA3E0F5308E55
:1027FC002F8D2E8C2D1217137BFF7A2479D0906994
:10280C0080E0FCA3E0FDA3E0FEA3E0F5308E2F8D6D
:10281C002E8C2D1217137BFF7A2479E6906984E0B5
:10282C00FCA3E0FDA3E0FEA3E0F5308E2F8D2E8CF3
:10283C002D1217137BFF7A2479FC906988E0FCA396
:10284C00E0FDA3E0FEA3E0F5308E2F8D2E8C2D1233
:10285C0017137BFF7A25791290698CE0FCA3E0FDBD
:10286C00A3E0FEA3E0F5308E2F8D2E8C2D121713C6
:10287C007BFF7A257928906990E0FCA3E0FDA3E02A
:10288C00FEA3E0F5308E2F8D2E8C2D1217137BFFAF
:10289C007A25793E906994E0FCA3E0FDA3E0FEA3C9
:1028AC00E0F5308E2F8D2E8C2D1217137BFF7A2591
:1028BC007954906998E0FCA3E0FDA3E0FEA3E0F559
:0B28CC00308E2F8D2E8C2D1217132242
:1043E500E4906BD4F01247FE906BD5EFF0C3943098
:1043F5004006E0D394394007906BD5E0B42E169073
:104405006BD5E0FF906BD4E02405F582E43461F5CB
:1044150083EFF08011906BD4E02405F582E43461DC
:10442500F583E4F0800C906BD4E004F0E0D39410B5
:1044350040B3752900752A00752B007B017A6179D7
:044445000512437F9A
:014449002250
:102AC000E490689FF07E257F6A123F34EF4E601BD2
:102AD0001247FE8F25E525B4310690689F740AF0F1
:102AE000E525B4320690689F7464F07E257F7012ED
:102AF0003F34EF4E600B12450D906ABC120F1580EB
:102B00000A906ABC120F2100002580906ABCE0F890
:102B1000A3E0F9A3E0FAA3E0FB7F007E8C7D0A7CB2
:102B200000120E64120EF6906AC2EEF0A3EFF0E40B
:102B30007B0AFAF9F8906ABCE0FCA3E0FDA3E0FE92
:102B4000A3E0FF120E64A804A905AA06AB07E47F60
:102B5000507EC3FDFC120E648E5C8F5D7E257F76F9
:102B6000123F34EF4E600A12450D9068A0EFF080DE
:102B700005E49068A0F07E257F7C123F34EF4E6024
:102B80000D12450D906AC0EEF0A3EFF0800A906A36
:102B9000C07401F0A374F4F07E257F82123F34EFFD
:102BA0004E600D12450D9068A3EEF0A3EFF0800784
:102BB000E49068A3F0A3F07E257F88123F34EF4EA7
:102BC000600A12450D906928EFF08006906928741C
:102BD00001F0E4F525E52575F008A4244CF582E420
:102BE0003426AF82FE123F34EF4E60171243E5E504
:102BF0002525E025E0246CF582E43469F583120F85
:102C0000158016E52525E025E0246CF582E434697D
:102C1000F583120F213F8000000525E525C3940CA4
:102C200040B3E4F568F569856982856883A37455C6
:102C3000F0856982856883A3A3F0856982856883AE
:102C4000A3A3A3F0906928E0FFE5692404F582E4DA
:102C50003568F583EFF0EFF4FFE5692405F582E4CC
:102C60003568F583EFF0E5692406F582E43568F50B
:102C7000837401F0E5692407F582E43568F583740F
:102C800055F08569828568837407F0E582241AF51A
:092C900082E43583F583E4F0FFD2
:012C99002218
:1042AE0043AB01C2E8C2EAE4FFEFC454F0F5B1C378
:1042BE00EF64809488500575B3D08003E4F5B3E4C1
:1042CE00F5B275BCC8F5BDF5BE75BF7875C4FFF502
:1042DE00C5F5C675C778F5A3F5A3F5A3F5A3F5A3A4
:1042EE00F5A3F5A3F5A30FBF0EBF90689FE0FF25C2
:1042FE00E0F5B475B50C75B66C75A11275AB02759B
:08430E00C13E75C3FF75C20337
:014316002284
:1044AD0075B180E4F5B3F5B2854CBCE54D5403FF11
:1044BD0033333354F8FFE54D54E04FFFE54EC4134D
:1044CD0054074FF5BDE54E33333354F8FFE54FC474
:1044DD001354074FF5BEE54F33333354F8F5BF850D
:1044ED0051A38552A38553A38554A38555A3855602
:1044FD00A38557A38558A3E550540F2450F5B32237
:10313600E59B541F6020200B1A7E257F8E12353E9C
:10314600E59B541FFF7E007D0312370C7E257F987A
:1031560012353EE4F59BE5BA30E008E4F5B375B107
:1031660080F5B2E5CFF47003023240752701E4F52D
:1031760026E5CFF45527700302322EE526C454F017
:10318600F5B1E5B2547F6420706FE5B3540FF55086
:1031960085BC4CE5BD541FFF131313541FFFE5BD3B
:1031A60054E044184FF54DE5BDC43354E0FFE5BE89
:1031B600131313541F4FF54EE5BEC43354E0FFE519
:1031C600BF131313541F4FF54F85A35185A3528583
:1031D600A35385A35485A35585A35685A35785A3D5
:1031E60058E4F5B2E54C547EB54C0575B3508003F2
:1031F60075B3D0E5502405FF22E5B2549F60232025
:103206000B207E257F9B12353EAFB27E007D0312DA
:10321600370CAFB37E007D0312370C7E257FA612D6
:10322600353EE4F5B275B3D0E52725E0F52705264A
:0C323600E526C3940850030231777F00A6
:013242002269
:10423400C219E4F562F50BD296F561F563FF7F4090
:1042440090692BE4F0A3DFFC7F40E4F564F56A1287
:104254002AC01242AEC2ADE4F5C9D2CDD2CCC2C995
:10426400C2CAF5CDF5CC906AC2E0F5CBA3E0F5CA9D
:1042740085CBCD85CACCE4F598D29E438740C29FB6
:10428400C2ACC298C29975B81075B710D2CAD29C84
:10429400D2AC124716C2D9E5E92464F5EB30D7064F
:0942A400E5F904F5FB2285F9FBA4
:0142AD0022EE
:01484E002247
:01484F002246
:05001E00D29CD2AC22CF
:014850002245
:10466600E4F568F569E5692401FFE43568F5838FAB
:104676008263A201906A9C63A2017F081229B28517
:104686006982856883E0F561E4F563D290C291C2E0
:1046960096D299200B0D7E257FA87C6A7D9CAB6106
:0446A6001232432267
:103D0C00E56AC394404003E4F56A742B256AF58296
:103D1C00E43469F583E0FF30E16F742B256AF5829A
:103D2C00E43469F583EF54FDF0E4906475F0A3740A
:103D3C000DF090667AE0906477F0A37419F0A37498
:103D4C0048F0A37479F0E56A131313541FFF9068BD
:103D5C00A0E02F90647BF0E56A540725E025E02471
:103D6C0080A3F0A37408F0F5F0E56AA4249FF58213
:103D7C00E5F03466F58363A20190647E63A2017F53
:0E3D8C00081229B2056A7F0122056A7F002213
:014851002244
:101F66003000469080E8E0700F12444A300D077E3C
:101F7600257FB112353EC21A9080E8E0B40E129069
:101F860080037408F0300D077E257FBA12353EC2F5
:101F96001A9080E8E0B4060F201A0C300D077E2553
:101FA6007FC512353ED21AC200201A0302206820CD
:101FB60019071237ED8F258003E4F525E5256047DF
:101FC600300D0C7E257FDB7C6A7DC8FB123243E533
:101FD600E92410F5EB30D708E5F92428F5FB80064F
:101FE600E5F92427F5FB906AC863A201906A9C6311
:101FF600A201AF251229B2852561E4F563D290C20C
:1020060091D219C296D29920D90302233DC2D9E5AD
:10201600E92410F5EB30D708E5F92428F5FB80060E
:10202600E5F92427F5FBE562D39400500302233D2E
:10203600C291856267E4F56290699C63A201906A29
:10204600C863A201AF671229B2AF6712344E200DE2
:102056000302233D7E257FE07C6A7DC8AB67123292
:102066004322742B2564F582E43469F583E020E08D
:10207600020564E564C394404003E4F56412313616
:10208600EF6069E54F640F70639068A0E0FF654EEE
:10209600705A742B2564F582E43469F583E0FE30CA
:1020A600E04A742B2564F582E43469F583EE54FE28
:1020B600F0754C48754D79E564131313541FFEEF04
:1020C6002EF54EE564540725E025E02480F54F758E
:1020D600500875F008E564A4249FF582E5F034669F
:1020E600F5837D517F081229A91244AD300202C240
:1020F6000220D90302233DC2D9E55B60030222CB4D
:10210600E562D3940050030222CBC291856267E454
:10211600F562200B0D7E257FE57C697D9CAB671201
:102126003243E56764586010300B030222CB7E25EC
:102136007FED12353E0222CBE4F525E52525E02587
:10214600E024BEF582E43469F583E09068A9F0E501
:102156002525E025E024BFF582E43469F583E09087
:1021660068A8F0E52525E025E024C0F582E4346979
:10217600F583E09068A7F0E52525E025E024C1F584
:1021860082E43469F583E09068A6F0200B0B7E2587
:102196007FF6E4FBFDFC123243E52525E025E0242D
:1021A6006CF582E43469F583E0FCA3E0FDA3E0FE70
:1021B600A3E0FF9068A6E0F8A3E0F9A3E0FAA3E0A5
:1021C600FB120853123B1E8F338E328D318C3075C5
:1021D6002DFF752E25752FFC7B017A6879AA1217BB
:1021E6000D7B017A6879AA123BCE8E658F66200B2D
:1021F60058752DFF752E25752FFF9068A6E0FCA358
:10220600E0FDA3E0FEA3E0F5338E328D318C30E5A0
:102216002525E025E0246CF582E43469F583E0FCAD
:10222600A3E0FDA3E0FEA3E0F5378E368D358C34B2
:10223600AC65AD66EC12095E8F3B8E3A8D398C38F3
:102246007B017A6879AA12170D200B22752DFF756E
:102256002E26752F23AC65AD66EC12095E8F338E84
:10226600328D318C307B017A6879C812170D200BBC
:102276000B7E687FAA7B057D321238C975F002E5B0
:1022860025A4249FF582E5F03466F583E566F0E53E
:1022960065FF3395E075F002E525A424A0F582E5F7
:1022A600F03466F583EFF0E5251313543F242BF540
:1022B60082E43469F5837403F00525E525C3940C9F
:1022C6005003022141E55B7042E5E92410F5EB304D
:1022D600D708E5F92428F5FB8006E5F92427F5FB60
:1022E60090692AE004F07006906929E004F090688D
:1022F600A3E0FEA3E0FFD390692AE09F906929E05E
:102306009E4034755B01E4F0A3F022E4F55BE561E1
:10231600600B741C2569F569E43568F568E5E92400
:1023260010F5EB30D708E5F92428F5FB8006E5F92A
:072336002427F5FB124666A7
:01233D00227D
:03484A007F0022CA
:10085300EC4D6011E8497017ED33EC3304600DE49F
:10086300FCFFFEFD22E933E8330470F80209CC12E1
:10087300099758046009E4CC2481500628500902E2
:1008830009D62840030209D3C0E0EB4A7044B9807B
:1008930006D0E0FB0209C2EF4E701CBD8008EBFFDF
:1008A300EAFEE9FD80EBE98DF0A4FEE5F002093CE8
:1008B300E9CDF9EAFEEBFFEF89F0A4FCE5F0CE8980
:1008C300F0A42EFFE435F0CD89F0A42DFEE435F03D
:1008D3008067EF4E7005BD80D780C3EF8BF0A4AC6B
:1008E300F0EE8BF0A42CFCE435F0F8EF8AF0A42CA6
:1008F300E5F038FCE433CB8DF0A42CFCE5F03BF8B9
:10090300EE8AF0A42CFCE5F038F8E433CF89F0A4A8
:100913002CFCE5F038CF3400CE89F0A42FFFE5F0AE
:100923003EFEE433C98DF0A42EFEE5F039CD8AF006
:10093300A42FFFE5F03EFEE43DFD33D0E0FB50077E
:100943000BBB000F0209D6EC2CFCEF33FFEE33FE9A
:06095300ED33FD0209AEC8
:1009590075F020800E75F010800575F0087D007E19
:10096900007F003392D530D503120EF6EC334010D8
:10097900EF33FFEE33FEED33FDEC33FCD5F0ED2222
:0E098900E5F0247EA2D513CC92E7CDCEFF225E
:1016B100E541242DF8E6054122782A301702782DDC
:1016C100E475F001120F52020DD02010EB7F2ED2E3
:1016D100108018EF540F2490D43440D4FF30140BF1
:1016E100EF24BFB41A0050032461FFE542600215E4
:1016F100420545E5457002054430170D782AE47529
:10170100F001120F52EF020E1602461F7403D21798
:101711008003E4C217F5418B2A8A2B892CE4F54218
:10172100F544F545E54260077F201216EC80F5751A
:1017310043FFC211C210C212C213C215C216C2188F
:101741001216BAFF700D3017057F001216FDAF4556
:10175100AE4422B4255FC2D5C2141216BAFF24D0FA
:10176100B40A00501A75F00A784230D50508B6FF60
:101771000106C6A426F620D5047002D21380D9240E
:10178100CFB41A00EF5004C2E5D2140219EAD21103
:1017910080C6D21080C0D21280BCD2D580BAD215F8
:1017A10080B47F201216EC2012077401B54200406C
:1017B100F11216B1FF1216EC021725D218D21680BB
:1017C100951216B1FB1216B1FA1216B1F94A4B7005
:1017D1000679E17A1A7BFF20122EE542602A7E000B
:1017E1008E82758300120DE960060EEE654370F07E
:1017F100C2D5EBC0E0EAC0E0E9C0E0EE121A4AD07F
:10180100E0F9D0E0FAD0E0FB120DD0FF60AAEBC006
:10181100E0EAC0E0E9C0E01216ECD0E02401F9D022
:10182100E03400FAD0E0FBE5430460DCD543D98025
:1018310087D21280A2121A2D60F7E54370010412BB
:101841000B7DA943600DE543600914F543121AD4D9
:10185100EF60F3EA30E702F404C3995077EAF42524
:10186100430430E701E404F543800D121A2D60C1F1
:10187100EA05432543120B7DEA7840F630E701E49F
:10188100254304D5430420150114121A4AE4C0E08B
:10189100121AD47840E6601320E70714F61216D422
:1018A100802204F6D0E014C0E07F001216D4E54394
:1018B10060071216CB1543800B3015031216CBD0DF
:1018C100E0021725D0E00480C5121A2D60A0E5437F
:1018D10004120B7D7840EAF6E5432015026001040D
:0518E1002404121A4A64
:1018E60074FF04C0E0121AD41216D4E54320150280
:1018F60060031216CBD0E0B543E87F451216DE78BA
:1019060040E67F2B30E7047F2DF404C0E01216EC8E
:10191600D0E075F00A84C0F01216D5D0E01216D5C4
:10192600021725791080027908C216C2188008D2DB
:10193600D5790A8004790AC2D5E543047002F543D5
:10194600E4FAFDFEFF1216B1FC7B082011131216F5
:10195600B1FD7B1030100A1216B1FE1216B1FF7BD4
:1019660020EC3382D592D55013C3E43010069FFF86
:10197600E49EFEE42011039DFDE49CFCE4CBF8C24A
:1019860011EC700CCFCECDCCE824F8F870F38017AC
:10199600C3EF33FFEE33FEED33FDEC33FCEB33FBED
:1019A600994002FB0FD8E9EB301105F8D0E0C448A6
:1019B600B211C0E00AEC4D4E4F78207B0070C2EAAF
:1019C600B5430040BCC0E0121A4CD0F0D0E0201164
:1019D60004C4C0E0C4B211C0F01216D5D0F0D5F0E0
:1019E600EB021725120FB117C25319295817934C3A
:1019F600178F42192D4F19354419354917A8431920
:101A06003B55186C4618CA451836471B01501797A0
:101A16002D179B2E17BE2B179F2317BC201AEA2AB9
:101A2600175748000017B6E543B4FF03754306127F
:101A360016B1FC1216B1FD1216B1FE1216B1FF78E0
:101A460039020BAC790AA2D5201314301509B91046
:101A5600020404B9080104A2D5201602500104208C
:101A660012689212B542005034C0E07F203013193C
:101A76007F30A21272167215500F121AA3C212C22A
:101A860016C215C2187F30800F301503E9C0E01268
:101A960016EC301503D0E0F9D0E0B542CC3015177E
:101AA6007F30B9100C1216EC7F583014077F7880FF
:101AB60003B908031216EC3012057F2D0216EC7FCF
:101AC600202018F87F2B2016F322921280CF7F0059
:101AD600B4070050052439F8E6FF22286E756C6CB1
:101AE6002900D2111216B13011F8C211784230D540
:101AF6000108F60217572D504349581216B1240310
:101B0600B405004001E4901AFC931216DD743A12F3
:0A1B160016DDD213754204021929EE
:10437F00D2108B268A2789281243D9C0E0FF124812
:10438F0018D0E040F3123639401F7829E6FB08E6D3
:10439F00FA08E6F94A4B60107826E6C0E008E6C056
:1043AF00E008E6C0E0120F6222ECC0E0EDC0E0EEE4
:1043BF00C0E0EFC0E01243D9D0F0AFF0D0F0AEF0D4
:1043CF00D0F0ADF0D0F0ACF080BBE475F001782602
:0643DF00120F52020DD086
:103B1E008F298E288D278C2674FFFFFEFDFCAB2986
:103B2E00AA28A927A826C3120F04602C7F807E9690
:103B3E007D187C4BAB29AA28A927A826120AD96082
:103B4E000250157F807E967D187CCBAB29AA28A9C2
:103B5E0027A826120AD95009AF29AE28AD27AC26C0
:103B6E0022AF29AE28AD27AC26120B468F2D8E2CF8
:103B7E008D2B8C2AEC120959C8ECC8C9EDC9CAEEB6
:103B8E00CACBEFCBAF29AE28AD27AC261209E4E4A1
:103B9E00FBFAF9F8120AD9601A401874FF252DF5B0
:103BAE002DE52C34FFF52CE52B34FFF52BE52A34CF
:103BBE00FFF52AAF2DAE2CAD2BAC2AEC12095922F3
:10099700E9D2E7C933E833F892D5EDD2E7CD33ECA6
:0709A70033FC5002B2D5221F
:1009AE00EC30E7100FBF000C0EBE00080DBD0004AA
:1009BE000BEB6014A2D5EB13FCED92E7FD2274FF56
:1009CE00FCFDFEFF22E480F8A2D574FF13FC7D80AF
:0309DE00E480EFC3
:1009E1000209CCE86480F8E933E83360110460F06F
:1009F100ED33EC337009E8FCE9FDEAFEEBFF22047C
:100A010060DED3EB9FEA9EE99DE8C2E78CF0C2F776
:100A110095F0400CE8CCF8E9CDF9EACEFAEBCFFB42
:100A210012099785D0F05804700320D5B3E80470FB
:100A3100075002B2D50209D692D5EC0460F7E4CC96
:100A4100C0E0C398F8603B94186008400DD0E0FB0B
:100A51000209AEE4FBFAC9FC8028E830E406E4C9E7
:100A6100FBE4CAFCE830E305E4C9CACBFCE854075F
:100A71006010F8C3E913F9EA13FAEB13FBEC13FC6A
:100A8100D8F130F52FC3E49CFCEF9BFFEE9AFEED0D
:100A910099FDD0E0FBEF4E4D4C701222DB030209B1
:100AA100D3EC2CFCEF33FFEE33FEED33FDED30E7FD
:100AB100EB0209AEEF2BFFEE3AFEED39FDD0E0FB84
:100AC10050130BBB00030209D6ED13FDEE13FEEF2D
:080AD10013FFEC13FC0209AE57
:100AD90074F8CC6480CCC86480C8F582046043C3D0
:100AE900EB9FF5F0EA9E42F0E99D42F0E89C45F063
:100AF90060305018E5825FFFE582F42B5582FB5088
:100B0900210ABA001D09B90019088016E5825BFBA4
:100B1900E582F42F5582FF50090EBE00050DBD0078
:100B2900010CC3EB9FF5F0EA9E42F0E99D42F0E823
:0D0B39009C45F06007CC4820E701B3EC229A
:100B4600EDD2E7CD33EC3392D524814006E4FFFEA7
:100B5600FDFC22FCE4CFCECDCC24E0501174FF8006
:100B6600EDC3CC13CCCD13CDCE13CECF13CF0470A3
:070B7600F030D5DE020EF69F
:100B7D00F920E72824F950037907E4F42402FB183F
:100B8D00DBFDE624FB5014E9600DE4F618E604F6EF
:0F0B9D00B40A08E4F6D9F57401F60A22C2D5228B
:100BAC00ED33EC3392D5FA602AB4FF33EDC2E77B18
:100BBC00FF60067A0B79D1E4227A0B79DA20D5041E
:100BCC007A0B79D5224E614E002B494E46002D49A9
:100BDC004E4600E47A08F608DAFC7B00740722E83B
:100BEC00C0E0ECC0E0EDC0E0EEC0E0EFC0E0EA75C4
:100BFC00F010A4CAABF075F04DA42BFBE435F0FC5F
:100C0C00EA2410FAEB34C5FBEC34D9FCEDC2E7FF57
:100C1C0075F056A4F42411C5F0F434C58FF0A42A51
:100C2C00E5F03BE43CF620E714120D90D0E0FFD049
:100C3C00E0FED0E0FDD0E0FC120CB28014F4041203
:100C4C000D90D0E0FFD0E0FED0E0FDD0E0FC12082B
:100C5C0053D0E0F8E6FAEDD2E7CD33EC332482FB47
:100C6C00E4C3CF33CFCE33CECD33CD33DBF37B07E1
:100C7C0075F00A846004F6081B0AE5F0F6088FF09C
:100C8C00740AA4FFACF08EF0740AA42CFEACF050E5
:100C9C00010C8DF0740AA42CFDE435F0F608DBDEB3
:030CAC00740722A8
:10362600C211C212C213C214F9E4F52CF52DFCFD29
:10363600FEFFE91010EA20130CB42D04D213D32296
:10364600B42B02D32224D0504794095041240A3087
:103656001415F8852DF0740AA42872E74051C5F0B8
:10366600704D85F02DD322D212C0E0E4FBFA79200A
:103676007841120853ECF8EDF9EEFAEFFBD0E0FCD6
:10368600E41209631209E83011B4152CD322240A76
:10369600201420B4FE0720111AD211D32224EB6085
:1036A6000424E0700EA2139211D214C213D322C3C3
:1036B6000209CCE430140BE52D301302F404A211F8
:1036C60092133012EA252C20D2E5A2E7921450027A
:1036D600F404B4260050D8CCC0E0EDC0E0EEC0E063
:1036E600EFC0E0EC120D90D0E0FFD0E0FED0E0FDA0
:1036F600D0E0FC2014051208538003120CB23013DC
:0637060003120D4FC32267
:100CAF000209D6EC5D046005E8590470030209CC13
:100CBF00120997580460F6EC4860F2EC7004FDFEE0
:100CCF00FF22C860DB2481C85009C3986002500618
:100CDF000209D39850CAF582E9294B4A7005AB82B5
:100CEF000209C275F0007C1A7880C3EF9BEE9AED73
:100CFF0099400DC3EF9BFFEE9AFEED99FDE842F090
:100D0F00DC23ACF0D0E0FFD0E0FED0E0FDAB8220E2
:100D1F00E7101BEB60BAEC2CFCEF33FFEE33FEED6C
:100D2F0033FD0209AEE803F830E705C0F075F000B7
:100D3F00EF2FFFEE33FEED33FD40B830E7C280AA50
:100D4F00ED33EC33600A047003BD8004ECB2E7FCB2
:010D5F002271
:100D60003F8000004120000042C80000447A00009B
:100D7000461C400047C35000497424004B1896801D
:100D80004CBEBC205A0E1BCA6753C21C749DC5AE14
:100D9000FB60065407601C2323120DBEEB54386021
:100DA00009120DAA120DB9120853ECF8EDF9EEFA7A
:100DB000EFCB22EB120DB980F1543803241C900DB7
:100DC00060FE93FC0EEE93FD0EEE930ECE93FF228B
:103DA600021053E493A3F8E493A34003F68001F2D0
:103DB60008DFF48029E493A3F85407240CC8C3331E
:103DC600C4540F4420C8834004F456800146F6DFED
:103DD600E4800B01020408102040809047E2E47E54
:103DE600019360BCA3FF543F30E509541FFEE493E2
:103DF600A360010ECF54C025E060A840B8E493A3A9
:103E0600FAE493A3F8E493A3C8C582C8CAC583CAD3
:103E1600F0A3C8C582C8CAC583CADFE9DEE780BE8B
:0147FD0000BB
:100DD000BB010689828A83E0225002E722BBFE0221
:090DE000E32289828A83E4932254
:100DE900BB010CE58229F582E5833AF583E02250BF
:100DF90006E92582F8E622BBFE06E92582F8E22209
:0D0E0900E58229F582E5833AF583E4932222
:100E1600BB010689828A83F0225002F722BBFE01BB
:020E2600F322B5
:100E280075F008758200EF2FFFEE33FECD33CDCC81
:100E380033CCC58233C5829BED9AEC99E582984004
:100E48000CF582EE9BFEED9AFDEC99FC0FD5F0D6E1
:100E5800E4CEFBE4CDFAE4CCF9A88222B800C1B90B
:100E68000059BA002DEC8BF084CFCECDFCE5F0CB49
:100E7800F97818EF2FFFEE33FEED33FDEC33FCEB82
:100E880033FB10D703994004EB99FB0FD8E5E4F93D
:100E9800FA227818EF2FFFEE33FEED33FDEC33FC2A
:100EA800C933C910D7059BE99A4007EC9BFCE99A1E
:100EB800F90FD8E0E4C9FAE4CCFB2275F010EF2F63
:100EC800FFEE33FEED33FDCC33CCC833C810D70763
:100ED8009BEC9AE899400AED9BFDEC9AFCE899F89E
:0E0EE8000FD5F0DAE4CDFBE4CCFAE4C8F92231
:0E0EF600C3E49FFFE49EFEE49DFDE49CFC220D
:100F0400EB9FF5F0EA9E42F0E99D42F0E89C45F043
:010F140022BA
:0C0F1500ECF0A3EDF0A3EEF0A3EFF0224F
:100F2100A8828583F0D083D082120F38120F381235
:100F31000F38120F38E473E493A3C583C5F0C5835A
:100F4100C8C582C8F0A3C583C5F0C583C8C582C81A
:010F5100227D
:100F5200FAE6FB0808E6F925F0F618E6CA3AF622A0
:100F6200BB011A89828A83D0F0D0E0F8D0E0F9D0B0
:100F7200E0FAD0E0FBE8C0E0C0F00210415016E910
:100F8200F8D083D082D0E0F9D0E0FAD0E0FBC08282
:100F9200C083021038BBFE16E9F8D083D082D0E0BD
:0F0FA200F9D0E0FAD0E0FBC082C08302104A22EF
:100FB100D083D082F8E4937012740193700DA3A3CF
:100FC10093F8740193F5828883E4737402936860E3
:060FD100EFA3A3A380DFE3
:10481800EFC394094005EF940E4003BF2003D380F3
:0348280001C322A7
:102C9A008B268A278928E4F532F531F530F52FF5A8
:102CAA002DF52EE52A452B45296012EBC0E0EAC036
:102CBA00E0E9C0E0AB29AA2AA92B120F62AB2605CC
:102CCA0028E528AA277002052714F9120DD0F53332
:102CDA00C394094007E533D3940D40E1E5336420FA
:102CEA0060DBE533B42D05432E038016E533B42BA0
:102CFA0005432E01800C74FF2528F52874FF35271B
:102D0A00F527E52C60046410703FAB26AA27A92892
:102D1A00120DD064306009E52C702E752C0A8029BA
:102D2A00900001120DE9FF64786004EFB458134370
:102D3A002E01752C1074022528F528E43527F5276D
:102D4A008007E52C7003752C08AB260528E528AA10
:102D5A00277002052714F9120DD0F533C394614088
:102D6A000AE533D3947A50035333DF74D02533F50D
:102D7A0033C3940A400CE5339411406D74F925333A
:102D8A00F533E533D3952C5060432E0185323785D0
:102D9A003136853035852F34AF2C7E00E4FCFDAB0F
:102DAA0032AA31A930A82F120FE9C8ECC8C9EDC957
:102DBA00CAEECACBEFCBE4FCFDFEEB2533F532EECF
:102DCA003AF531ED39F530EC38F52FAF32AE31AD99
:102DDA0030FCAB37AA36A935A834D3120F045003F6
:102DEA00022D53432E04022D53E52E20E003E480E6
:102DFA002DE52A452B4529601EAB26E52824FFF937
:102E0A00E52734FFFAEBC0E0EAC0E0E9C0E0AB290D
:102E1A00AA2AA92B120F62E52E30E20774FFFFFEE1
:102E2A00FDFC22E52EAF32AE31AD30AC2F30E103DE
:042E3A00020EF6226C
:103BCE008B268A278928AB26AA27A928120DD0FF73
:103BDE00124818500D74012528F528E43527F527CD
:103BEE0080E4D210AB26AA27A928120DD0FF642B91
:103BFE006004EFB42D1BAB260528E528AA2770021A
:103C0E00052714F9120DD0642D6003D38001C392E1
:103C1E0010E4F529F52AAB26AA27A928120DD0FF04
:103C2E0012483B5036AB26AA27A928120DD0FF33D7
:103C3E0095E0FEEF24D0FBEE34FFFAAE29AF2A7CDE
:103C4E00007D0A120FD7EF2BF52AEE3AF5297401F3
:103C5E002528F528E43527F52780BB301006AE2938
:0E3C6E00AF2A8009C3E4952AFFE49529FE22BF
:100FD700EF8DF0A4A8F0CF8CF0A428CE8DF0A42E2E
:020FE700FE22E8
:100FE900E88FF0A4CC8BF0A42CFCE98EF0A42CFCA7
:100FF9008AF0EDA42CFCEA8EF0A4CDA8F08BF0A425
:101009002DCC3825F0FDE98FF0A42CCD35F0FCEB83
:101019008EF0A4FEA9F0EB8FF0A4CFC5F02ECD3948
:0F102900FEE43CFCEAA42DCE35F0FDE43CFC22B5
:09103800EBF608EAF608E9F622DD
:09104100EBF0A3EAF0A3E9F022B0
:09104A00EBF208EAF208E9F222D7
:0F483B00EFC394304007EF943A50028001C3223C
:00000001FF
